:020000040000FA
:100000006C2800000000000009001108820760341D
:100010003134323433346134343435343634623448
:1000200037343834393463342A3430342334643444
:100030001C3084008901831608148312080880008C
:10004000840A890A28300402031D1B2808001C307A
:1000500084008901000888008316081208155530AD
:100060008900AA30890088148312000000008316DA
:10007000081E34288312840A890A28300402031DCA
:100080002A2808008D0050308E008E0B45288D0BDD
:100090004328080090008615033042208611033063
:1000A0004220900B4B280800910104309200FE3052
:1000B0006500A0304220060E940004309300910A9F
:1000C000940C031C0528930B5F2803148316850DDD
:1000D0008312920B592800348501030165008601C3
:1000E000F0306600831681138312F0304A20182006
:1000F000860101309500A1201C30E020031D7828E6
:100100002A301102031996281508013C031D912875
:100110000430860096308F00C83042208F0B8C2828
:1001200078280130860096308F008C2002308600BF
:10013000A1200421A1201C30E020031D75282720C8
:100140007828A801030165000608F039F03A031D7C
:10015000A228F0304220060808308B0063005420AB
:10016000FF3991000319A228F030422006302802FE
:10017000031DCD28D920031DC12840304A20110875
:1001800008002A308400000884038000840A840A5E
:100190002F300402031DC328A803D9200319A12866
:1001A00040304A2029302807840011088000A80A1E
:1001B000A22823301102031908002A301102080076
:1001C000AF00A8010230B100F228150A95000630F0
:1001D000AF07A801B10BF22855304220F0304A2079
:1001E000031108002930280784000008B0002F08F8
:1001F0002807840000083002031DE528A80A0630FD
:100200002802031DF2280800A801293028078400CD
:100210000008B0002F082807840030088000A80AD2
:0A02200006302802031D052908001E
:02400E00F23F7F
:104200003100320033003400350036003100320016
:084210003300340035003700D3
:00000001FF
